:100000000C942A000C9472000C9496000C944500F9
:100010000C9445000C9445000C9445000C9445004C
:100020000C9445000C9445000C9445000C9445003C
:100030000C9445000C9445000C9445000C9445002C
:100040000C9445000C9445000C9445000C9445001C
:100050000C94450011241FBECFE5D8E0DEBFCDBF14
:1000600010E0A0E6B0E0E2E4F2E002C005900D92FC
:10007000A037B107D9F710E0A0E7B0E001C01D92AA
:10008000A537B107E1F70C94EB000C9400001CBEFF
:1000900013BC8DE683BF85BD089510927400109245
:1000A000730085E085BF80EC8BBF089540B34C7032
:1000B00080917200482BE0E6F0E0E40FF11D8081B2
:1000C000992787FD90952091730030917400820FDD
:1000D000931F9093740080937300469546954093C8
:1000E000720008951F920F920FB60F9211242F9352
:1000F0003F934F935F936F937F938F939F93AF93B0
:10010000BF93EF93FF930E945600FF91EF91BF9131
:10011000AF919F918F917F916F915F914F913F919F
:100120002F910F900FBE0F901F9018951F920F9256
:100130000FB60F9211242F933F934F935F936F93BA
:100140007F938F939F93AF93BF93EF93FF930E94FF
:100150005600FF91EF91BF91AF919F918F917F9149
:100160006F915F914F913F912F910F900FBE0F9024
:100170001F901895882311F46CBF0895813009F001
:10018000089563BD08950895882311F4C09A0895D1
:10019000C09808950895CF93DF93EC0118161906BF
:1001A00054F460E0862F0E94BA0081E00E94C400EF
:1001B0006C2F81E00BC060E081E00E94BA0080E01B
:1001C0000E94C4008C2F8195682F80E00E94BA00A5
:1001D000DF91CF910895CFE5D8E0DEBFCDBF1ABA49
:1001E00089E087BB14BA80E881BB0E9447000E9467
:1001F0004D0078948091730090917400209170006C
:1002000030917100821B930BAA2797FDA095BA2FFE
:100210008F3F9105A105B10529F024F08FEF90E003
:10022000A0E0B0E081302FEF92072FEFA2072FEF71
:10023000B20724F481E09FEFAFEFBFEF0E94CB0045
:02024000D9CF14
:100242000001FF00FF000001010000FF00FF0100AC
:00000001FF
